:100000000C940E130C9438130C9438130C9438136E
:100010000C9438130C9438130C9438130C94381334
:100020000C9438130C9438130C9496D60C9413D764
:100030000C9438130C9438130C9438130C94381314
:100040000C9438130C94947A0C9438130C94381341
:100050000C9438130C9438130C94BD910C94F5D572
:100060000C9438130C9438130C9438130C943813E4
:100070000C9438130C9438130C9438130C943813D4
:100080000C9438130C9438130C9438130C943813C4
:100090000C943FCA0C94381384D3B0D3D2D3D2D3A8
:1000A000D2D3D2D3D2D3D2D3D2D3D2D3D2D3D2D328
:1000B000D2D3D2D3C8D3C0D3B8D3D2D3D2D3D2D34E
:1000C000D2D3D2D3D2D3D2D3AAD390D398D3A2D3DC
:1000D000084AD73B3BCE016E84BCBFFDC12F3D6CAF
:1000E00074319ABD56833DDA3D00C77F11BED9E415
:1000F000BB4C3E916BAAAABE000000803F05A84CF5
:10010000CDB2D44EB93836A9020C50B991868808C0
:100110003CA6AAAA2ABE000000803F004E414E49DC
:100120004E495459494E46CDCCCC3D0AD7233C17B5
:10013000B7D13877CC2B329595E6241FB14F0A0002
:100140000020410000C84200401C4620BCBE4CCAF2
:100150001B0E5AAEC59D742020506C616E6E657288
:1001600042756666657242797465733A200020466E
:10017000726565204D656D6F72793A2000436F6D31
:1001800070696C65643A204E6F76202039203230D9
:1001900031380A00207C20417574686F723A20283B
:1001A00044722E5068696C3344290A003230313869
:1001B0002D30382D303100204C617374205570641F
:1001C000617465643A2000312E312E390A004D6188
:1001D000726C696E0020536F66747761726520528D
:1001E000657365740A00205761746368646F6720E3
:1001F00052657365740A002042726F776E206F75C6
:10020000742052657365740A002045787465726EB7
:10021000616C2052657365740A00506F7765725582
:10022000700A0073746172740A005072696E7465AA
:10023000722068616C7465642E206B696C6C28296F
:100240002063616C6C6564210A004B494C4C454449
:100250002E20004B494C4C2063617573656420620D
:100260007920746F6F206D75636820696E616374A7
:100270006976652074696D65202D206375727265DD
:100280006E7420636F6D6D616E643A200020746F30
:100290006F206C6F6E6720657874727573696F6E0E
:1002A0002070726576656E7465640A0020636F6CF9
:1002B0006420657874727573696F6E2070726576EC
:1002C000656E7465640A006F6B00526573656E64D9
:1002D0003A2000416476616E6365204B3D003F4BE0
:1002E0002076616C7565206F7574206F6620726171
:1002F0006E67652028302D3130292E0A003A200003
:1003000050726F6265205A204F6666736574003FB5
:100310005A206F7574206F662072616E67652028A1
:100320002D3520746F203230290A00454550524F38
:100330004D204F4B0A00426564204C6576656C6920
:100340006E6720004661696C656420746F20656E7D
:1003500061626C6520426564204C6576656C696EEF
:10036000670A00426564204C6576656C20436F72B5
:1003700072656374696F6E204D61747269783A00BA
:100380004E6F2063617365206C696768740A00436F
:10039000290A0061626C656420286D696E207465AD
:1003A0006D702000436F6C642065787472756465AD
:1003B00073206172652000496E76616C6964206506
:1003C000787472756465720A0020643A0020693A94
:1003D0000020703A0050726F6265205A204F6666A6
:1003E0007365743A200020466C6F773A2000205ADB
:1003F00000205900580020204D61783A2000205AF2
:1004000000205900580020204D696E3A20004F66A8
:1004100066004F6E2000536F667420656E647374BF
:100420006F70733A20004F66667365747320617055
:10043000706C696564004572723A20546F6F206673
:1004400061722100546F6F206661722066726F6D59
:10045000207265666572656E636520706F696E7483
:100460000A00205400205200416363656C6572618C
:1004700074696F6E3A2050004D31343520533C6919
:100480006E6465783E206F7574206F662072616EB1
:1004900067652028302D31290A002F2F20003A00CF
:1004A0004361703A00544845524D414C5F50524FA1
:1004B00054454354494F4E004155544F5245504FB7
:1004C00052545F53445F53544154555300454D4576
:1004D0005247454E43595F504152534552004341A4
:1004E00053455F4C494748545F4252494748544E30
:1004F00045535300544F47474C455F4C4947485478
:100500005300534F4654574152455F504F57455241
:10051000004255494C445F50455243454E54004CAF
:100520004556454C494E475F44415441005A5F503F
:10053000524F4245004155544F4C4556454C005092
:1005400052494E545F4A4F420050524F4752455312
:1005500053004155544F5245504F52545F54454DEE
:100560005000564F4C554D45545249430045455057
:10057000524F4D0053455249414C5F584F4E5F58C2
:100580004F4646004649524D574152455F4E414DF8
:10059000453A4D61726C696E20312E312E3920281A
:1005A0004769746875622920534F555243455F432C
:1005B0004F44455F55524C3A68747470733A2F2F0C
:1005C0006769746875622E636F6D2F4D61726C6917
:1005D0006E4669726D776172652F4D61726C696EDE
:1005E0002050524F544F434F4C5F56455253494F42
:1005F0004E3A312E30204D414348494E455F5459C3
:1006000050453A3344205072696E746572204558E3
:100610005452554445525F434F554E543A3120553C
:100620005549443A34306365363164312D3265645E
:10063000302D343533302D383330342D3535653366
:1006400065656161656266660A00334420507269BF
:100650006E746572204F66662E0020573A00426520
:100660006420636F6F6C696E672E2E2E0042656486
:100670002068656174696E672E2E2E0020573A003F
:100680004520436F6F6C696E672E2E2E0045204803
:10069000656174696E672E2E2E006F6B004D3131CF
:1006A000332053004B494C4C45442E2000454348D1
:1006B0004F00494E464F004552524F52530044524C
:1006C0005952554E00434F4D4D554E4943415449A3
:1006D0004F4E006F666600AD06B206B706BE06C591
:1006E0000644454255473A0050726F74656374651D
:1006F000642050696E0A0000011C1D132FFFFFFFCC
:10070000FF1E1F12FF18FFFFFF20211124FFFFFF14
:10071000FFFFFFFF0E10FFFFFF22230DFFFFFF0E65
:10072000260F2C272569730025696D202569730024
:100730002569682025696D20256973002569642075
:100740002569682025696D20256973002569792050
:10075000256964202569682025696D202569730055
:100760005072696E742074696D653A20004E6F2076
:100770006D6F76652E00436C69636B20746F207219
:100780006573756D652E2E2E00205A3A2000205973
:100790003A200042656420583A20004731205A31FF
:1007A000302046373030300A473120583020593019
:1007B000204637303030000A0A426564204C6576A6
:1007C000656C20436F7272656374696F6E204D6152
:1007D000747269783A00202844525952554E2900C3
:1007E000473239204175746F20426564204C65762C
:1007F000656C696E67003F2856296572626F736584
:10080000206C6576656C20697320696D706C61750C
:100810007369626C652028302D34292E0A00536CD0
:100820006565702E2E2E0047322F4733206261649B
:1008300020706172616D65746572730A00496E762D
:10084000616C69642065787472756465720A004130
:1008500063746976652045787472756465723A20B0
:100860000020453A00205A3A0020593A00583A00F0
:100870002C20002C2000486F6D6520585920666997
:100880007273740A00486F6D65205859206669724A
:100890007374005761726E696E673A20486F6D69B4
:1008A0006E672042756D702044697669736F72209F
:1008B0003C20310A00020204627573793A207061AB
:1008C0007573656420666F7220696E7075740A00B6
:1008D000627573793A2070617573656420666F7212
:1008E00020757365720A00627573793A2070726FB1
:1008F00063657373696E670A0050726F62696E6731
:10090000206661696C65640A0050726F62696E6787
:10091000206661696C656400205A3A200020593ACB
:10092000200042656420583A2000486F6D652025FC
:10093000732573257320666972737400206669726B
:1009400073740A005A0059005800486F6D65200002
:1009500020496E76616C696420657874727564658F
:100960007220004B494C4C45442E200053544F50AC
:100970005045442E20005072696E74657220737465
:100980006F707065642064756520746F2065727285
:100990006F72732E204669782074686520657272C4
:1009A0006F7220616E6420757365204D393939206E
:1009B000746F20726573746172742E202854656D93
:1009C00070657261747572652069732072657365F4
:1009D000742E2053657420697420616674657220DA
:1009E00072657374617274696E67290A004E6F20B4
:1009F000436865636B73756D2077697468206C69F3
:100A00006E65206E756D6265722C204C617374206A
:100A10004C696E653A2000636865636B73756D2081
:100A20006D69736D617463682C204C617374204C24
:100A3000696E653A20004C696E65204E756D626581
:100A400072206973206E6F74204C617374204C693E
:100A50006E65204E756D6265722B312C204C617372
:100A600074204C696E653A20004D31313000656E5E
:100A70007175657565696E67202200FF01FF0000D2
:100A8000A0400000A040000000400000C84200005C
:100A9000C84200000343000000000000C8420000FC
:100AA00000000000C8420000C842000003430000EC
:100AB00000000000000000000000000048420000AC
:100AC000484200008040000000003A0A0020286DE3
:100AD0006D290020204D393030204B004C696E6567
:100AE000617220416476616E63653A0A0020204D90
:100AF000383531205A005A2D50726F6265204F668A
:100B0000667365740020440020490020204D333076
:100B1000312050005049442073657474696E6773C6
:100B20003A0A0020460020420020480020204D3193
:100B300034352053004D6174657269616C206865BD
:100B40006174757020706172616D65746572733A5D
:100B50000A0020204D3432302053004175746F203C
:100B6000426564204C6576656C696E673A0A0020C0
:100B70005A0020590020204D323036205800486F4E
:100B80006D65206F66667365743A0A002045002023
:100B90005A002059002058002054002053002020E3
:100BA0004D32303520510020453C6D61785F655FE6
:100BB0006A65726B3E0020583C6D61785F785F6AB1
:100BC00065726B3E20593C6D61785F795F6A657232
:100BD0006B3E205A3C6D61785F7A5F6A65726B3E4E
:100BE00000416476616E6365643A20513C6D696EC4
:100BF0005F7365676D656E745F74696D655F75734E
:100C00003E20533C6D696E5F666565647261746514
:100C10003E20543C6D696E5F74726176656C5F66F0
:100C2000656564726174653E0020540020520020A6
:100C3000204D323034205000416363656C65726131
:100C400074696F6E2028756E6974732F7332293A38
:100C500020503C7072696E745F616363656C3E2006
:100C6000523C726574726163745F616363656C3E6C
:100C700020543C74726176656C5F616363656C3EA1
:100C80000A00204500205A0020590020204D323013
:100C9000312058004D6178696D756D204163636541
:100CA0006C65726174696F6E2028756E6974732F3C
:100CB0007332293A0A00204500205A0020590020AA
:100CC000204D3230332058004D6178696D756D20AC
:100CD0006665656472617465732028756E697473E6
:100CE0002F73293A0A00204500205A00205900207D
:100CF000204D39322058005374657073207065722E
:100D000020756E69743A0A0020204D32303020443C
:100D1000300A0020204D32303020440020446973D6
:100D200061626C65640A0046696C616D656E742071
:100D300073657474696E67733A0020204D313439DD
:100D40002043203B20556E69747320696E204365F3
:100D50006C736975730A00202047323120202020EF
:100D60003B0048617264636F64656420446566613A
:100D7000756C742053657474696E6773204C6F6171
:100D80006465640A00DC050000DC050000DC050089
:100D900000102700000000FA420000FA420000A004
:100DA000400000C8410000A0420000A0420080FCBA
:100DB000440000C042290A002062797465733B2018
:100DC00063726320002073746F72656420736574AE
:100DD00074696E67732072657472696576656420E4
:100DE0002800202863616C63756C61746564292137
:100DF0000A0020213D2000454550524F4D204352CE
:100E000043206D69736D61746368202D20287374AD
:100E10006F7265642920002053697A653A20004981
:100E20006E6465783A2000204D61726C696E3D56A3
:100E30003535290A0028454550524F4D3D0045455E
:100E400050524F4D2076657273696F6E206D6973D5
:100E50006D617463682000290A00206279746573EB
:100E60003B20637263200053657474696E6773205E
:100E700053746F726564202800454550524F4D20D1
:100E80006461746173697A65206572726F722E0A8B
:100E9000004572726F722077726974696E67207490
:100EA0006F20454550524F4D210A006F70656E000E
:100EB000545249474745524544003A20007A5F6DF5
:100EC000696E00795F6D617800785F6D696E0052C0
:100ED00065706F7274696E6720656E6473746F708D
:100EE000207374617475730A00456E6473746F7057
:100EF0007320256320256320256320256300205A65
:100F00003A0020593A0020583A00656E6473746FB5
:100F10007073206869743A2000486F6D696E6720AD
:100F20006661696C656400556E6B6E6F776E2063E9
:100F30006F6D6D616E643A20220020746F6F206CBB
:100F40006F6E6720657874727573696F6E2070724A
:100F50006576656E7465640A0020636F6C64206555
:100F60007874727573696F6E2070726576656E74D1
:100F700065640A00FFFDFCFAF8F6F4F2F0EEECEA24
:100F8000E9E7E5E3E1E0DEDCDAD9D7D5D4D2D0CFAA
:100F9000CDCBCAC8C7C5C3C2C0BFBDBCBAB9B7B63E
:100FA000B4B3B2B0AFADACAAA9A8A6A5A4A2A1A0A3
:100FB0009E9D9C9A99989795949392908F8E8D8BE5
:100FC0008A8988878684838281807F7E7D7B7A7907
:100FD0007877767574737271706F6E6D6C6B6A6909
:100FE0006867666564636261605F5E5D5C5B5A59F9
:100FF00058585756555453525150504F4E4D4C4BD4
:101000004A4A4948474646454443424241403F3E9A
:101010003E3D3C3B3B3A3938383736353534333250
:10102000323130302F2E2E2D2C2B2B2A29292827F8
:101030002726252524232322212120201F1E1E1D93
:101040001C1C1B1B1A191918181716161515141322
:101050001312121111100F0F0E0E0D0D0C0C0B0AA6
:101060000A09090808070706060505040403030220
:1010700002010000000000010000000100008000EB
:10108000555555000000400033333300AAAA2A000A
:101090004992240000002000C7711C009999190092
:1010A000D1451700555515003BB1130024491200D6
:1010B00011111100000010000F0F0F00E3380E0097
:1010C00043790D00CCCC0C00C3300C00E8A20B001F
:1010D00064210B00AAAA0A00703D0A009DD80900ED
:1010E000427B090092240900DCD3080088880800AC
:1010F0001042080000000800F0C1070087870700C1
:1011000075500700711C07003EEB0600A1BC0600ED
:101110006990060066660600703E060061180600CB
:1011200017F4050074D105005BB00500B29005000E
:10113000627205005555050078390500B81E050096
:10114000050505004EEC040087D40400A1BD040091
:1011500090A7040049920400C17D0400EE690400D8
:10116000C7560400444404005C3204000821040013
:1011700041100400000004003FF00300F8E0030009
:1011800026D20300C3C30300CCB503003AA8030072
:101190000A9B0300388E0300C08103009F75030083
:1011A000D0690300505E03001D5303003448030060
:1011B000913D03003333030016290300381F030059
:1011C00097150300300C0300030303000BFA020021
:1011D00049F10200BAE802005CE002002DD80200EA
:1011E0002DD0020059C80200B0C0020031B902007F
:1011F000DAB10200AAAA0200A0A30200BC9C02006D
:10120000FA9502005C8F0200DF88020082820200F1
:10121000457C02002776020027700200436A020024
:101220007C640200D05E02003F590200C8530200F5
:101230006563686F3A004572726F723A00205A3ADD
:101240000020593A0020436F756E7420583A0023ED
:101250002C0000B8220000561800003A0F0000B819
:10126000080000B1040000710200003E01000024EB
:10127000F4D43050C38E20C2A24017828B7011125A
:101280007A910D816CD90AA861E108C75866076197
:101290005143061E4B5D05C145A7041A41110409BF
:1012A0003D9803713931034036DB0265339102D436
:1012B000305402802E1D02632CEE01752AC501B048
:1012C00028A001102781018F2564012B244B01E008
:1012D000223401AC211F018D200D01801FFC0084F0
:1012E0001EED00971DDF00B81CD200E61BC60020D3
:1012F0001BBC00641AB200B219A8000A19A0006A47
:10130000189900D117910040178B00B51684003151
:10131000167E00B31579003A157300C7146F005894
:10132000146A00EE1366008813630025135E00C77D
:10133000125B006C12570015125400C1115100705D
:10134000114F0021114B00D61049008D1047004667
:1013500010440002104200C00F4000800F3E0042C7
:101360000F3C00060F3B00CB0E3800930E37005C9D
:101370000E3500270E3400F30D3200C10D31009000
:101380000D3000600D2E00320D2D00050D2C00D902
:101390000C2B00AE0C2900850C29005C0C270035B5
:1013A0000C27000E0C2600E80B2400C40B2400A020
:1013B0000B23007D0B23005A0B2100390B21001851
:1013C0000B2000F80A1F00D90A1E00BB0A1E009D50
:1013D0000A1D00800A1D00630A1C00470A1B002C1E
:1013E0000A1B00110A1A00F7091A00DD091900C4C6
:1013F000091900AB091900920917007B091800634D
:101400000917004C09160036091600200916000AB3
:10141000091500F5081500E0081400CC081400B800
:10142000081400A4081400900813007D0812006B33
:10143000081300580812004608120034081100234F
:101440000811001208110001081100F0071000E057
:10145000071000D0071000C0071000B0070F00A150
:1014600007100091070E0083070F0074070F006537
:10147000070E0057070E0049070E003B070D002E10
:10148000070E0020070D0013070D0006070D00F9D9
:10149000060C00ED060D00E0060C00D4060C00C89A
:1014A000060C00BC060C00B0060C00A4060B00994C
:1014B000060C008D060B0082060B0077060B006CF5
:1014C000060B0061060A0057060B004C060A004294
:1014D000060A0038060A002E060A0024060A001A28
:1014E000060A001006090007060A00FD050900F4B7
:1014F000050900EB050900E2050900D9050900D03E
:10150000050900C7050900BE050900B5050800ADBD
:10151000050800A50509009C050800940508008C35
:10152000050800840508007C050800740508006CA7
:10153000050700650508005D050700560508004E13
:10154000050700470507004005080038050700317A
:101550000507002A050700230507001C05060016DD
:101560000507000F0507000805060002050700FB38
:10157000040600F5040700EE040600E8040600E295
:10158000040700DB040600D5040600CF040600C9EA
:10159000040600C3040600BD040600B7040600B13B
:1015A000040500AC040600A6040600A00405009B88
:1015B00004060095040500900406008A04050085D1
:1015C000040500800406007A040500750405007017
:1015D0000405006B04050066040500610405005C59
:1015E00004050057040500520405004D0405004899
:1015F000040500430405003E0404003A04050035D8
:10160000040500300404002C040500270404002312
:101610000405001E0404001A040400160405001149
:101620000404000D0404000904050004040400007F
:10163000040400FC030400F8030400F4030400F0B5
:10164000030400EC030400E8030400E4030400E0E6
:10165000030400DC030400D8030400D4030400D016
:10166000030400CC030400C8030300C503030024E3
:10167000F404D9201BC40C5C0E9804C4095F0265F5
:10168000077101F405F900FB04B30048048700C1A9
:101690000369005803550003034500BE023A008465
:1016A00002310053022A002902250004022000E42E
:1016B000011C00C8011900AF011700980114008433
:1016C000011300710110006101100051010E00436F
:1016D000010D0036010B002B010B0020010B001542
:1016E0000109000C01090003010800FB000800F3D8
:1016F000000800EB000700E4000600DE000600D84A
:10170000000600D2000600CC000500C7000500C29C
:10171000000500BD000400B9000400B5000400B1DC
:10172000000400AD000400A9000400A5000300A20D
:101730000003009F0004009B000300980003009535
:1017400000020093000300900003008D0002008B54
:10175000000300880002008600020084000300816C
:101760000002007F0002007D0002007B0002007981
:10177000000200770001007600020074000200728F
:10178000000100710002006F0002006D0001006C9A
:101790000002006A000100690002006700010066A3
:1017A00000010065000100640002006200010061A8
:1017B000000100600001005F0002005D0001005CAC
:1017C0000001005B0001005A0001005900010058AF
:1017D00000010057000100560001005500010054AF
:1017E00000010053000000530001005200010051AD
:1017F000000100500001004F0001004E0000004EAB
:101800000001004D0001004C0001004B0000004BA6
:101810000001004A000100490001004800000048A2
:10182000000100470001004600000046000100459D
:101830000000004500010044000100430000004397
:101840000001004200000042000100410000004190
:10185000000100400001003F0000003F0001003E89
:101860000000003E0001003D0000003D0001003C82
:101870000000003C0000003C0001003B0000003B79
:101880000001003A0000003A000100390000003970
:101890000001003800000038000000380001003767
:1018A000000000370001003600000036000000365E
:1018B0000001003500000035000000350001003453
:1018C0000000003400000034000100330000003349
:1018D000000000330001003200000032000000323E
:1018E0000001003100000031000000310001003033
:1018F00000000030000000300001002F0000002F29
:101900000000002F0000002F0001002E0000002E1C
:101910000000002E0001002D0000002D0000002D11
:101920000000002D0001002C0000002C0000002C05
:101930000000002C0001002B0000002B0000002BF9
:101940000000002B0001002A0000002A0000002AED
:101950000000002A000100290000002900000029E1
:1019600000000029000000290001002800000028D4
:1019700000000028000000280000002800010027C7
:1019800000000027000000270000002700000027BB
:1019900000010026000000260000002600000026AE
:1019A00000000026000100250000002500000025A1
:1019B0000000002500000025000000250001002493
:1019C0000000002400000024000000240000002487
:1019D000000100230000002300000023000000237A
:1019E000000000230000002300000023000100226B
:1019F000000000220000002200000022000000225F
:101A00000000002200010021000000210000002150
:101A10000000002100000021000000210000002142
:101A20000001002000000020000000200000002035
:101A30000000002000000020000000200000002026
:101A40000001001F0000001F0000001F0000001F19
:101A50000000001F0000001F0000001F0001001E0A
:101A60000000001E0000001E0000001E00000029F3
:101A70000A002028002920453A0020280029205A61
:101A80003A002028002920593A0020280020583AFE
:101A900000537465707065722063757272656E7440
:101AA0002076616C75657320696E20252028416D54
:101AB0007073293A0A002042403A0020403A002040
:101AC0002F00546865726D616C2052756E6177618C
:101AD0007900453120544845524D414C2052554ED5
:101AE000415741590042454420544845524D414CCC
:101AF0002052554E41574159004B494C4C45442EBC
:101B00002000202D20496E76616C69642065787410
:101B10007275646572206E756D62657220210A00AF
:101B200048656174696E67206661696C656400422E
:101B300065642068656174696E67206661696C65BB
:101B4000640048656174696E67206661696C6564EC
:101B50000045312048656174696E67206661696C73
:101B60006564004D494E54454D5020747269676755
:101B700065726564004531204572723A204D494EC8
:101B800054454D50004572723A204D494E54454DD2
:101B90005020424544004D415854454D50207472E8
:101BA00069676765726564004531204572723A2045
:101BB0004D415854454D50004572723A204D4158A0
:101BC00054454D5020424544006265640A002C2073
:101BD00073797374656D2073746F70706564212000
:101BE0004865617465725F49443A20002CFFFFFF2D
:101BF000FFFF00010101010123646566696E652034
:101C000044454641554C545F4B642000236465664F
:101C1000696E652044454641554C545F4B69200030
:101C200023646566696E652044454641554C545FA2
:101C30004B702000504944204175746F74756E6577
:101C40002066696E6973686564212050757420741C
:101C50006865206C617374204B702C204B69206187
:101C60006E64204B6420636F6E7374616E747320B6
:101C700066726F6D2062656C6F7720696E746F207D
:101C8000436F6E66696775726174696F6E2E680A5C
:101C900000504944204175746F74756E652066610B
:101CA000696C6564212074696D656F75740A0054F0
:101CB0006865726D616C2052756E6177617900455F
:101CC0003120544845524D414C2052554E415741C8
:101CD000590048656174696E67206661696C656466
:101CE0000045312048656174696E67206661696CE2
:101CF000656400504944204175746F74756E6520A9
:101D00006661696C6564212054656D7065726174EB
:101D100075726520746F6F20686967680A00204BD0
:101D2000643A2000204B693A2000204B703A200092
:101D30000A20436C617373696320504944200A0090
:101D40002054753A2000204B753A2000206D6178B0
:101D50003A2000206D696E3A200020643A2000206D
:101D6000626961733A2000504944204175746F7470
:101D7000756E652073746172740A00504944204185
:101D800075746F74756E65206661696C6564212079
:101D9000426164206578747275646572206E756D39
:101DA0006265720A001000C90210012C0140012274
:101DB0000170011801B0010E01F00104015002FA96
:101DC00000B002F0003003E600D003DC009004D243
:101DD000007005C800A006BE000008B400B009AA43
:101DE00000D00BA000600E960060118C00001582E0
:101DF0000020197800C01D6E00A0226400B0275A90
:101E000000902C500000314600E0343C0010383285
:101E100000903A2800603C1E00A03D1400803E0A5D
:101E200000203F000070012C0190012701B0012229
:101E300001C0011D01F00118011002130130020E52
:101E4000016002090190020401C002FF000003FAD0
:101E5000004003F5008003F000D003EB002004E60F
:101E6000007004E100E004DC004005D700C005D2AA
:101E7000004006CD00D006C8008007C3003008BE71
:101E800000F008B900C009B400B00AAF00B00BAA56
:101E900000D00CA500000EA000500F9B00C01096B3
:101EA000005012910000148C00C0158700B01782FA
:101EB00000B0197D00D01B7800001E730040206E1A
:101EC0000090226900F024640040275F0090295AA6
:101ED00000E02B5500102E500020304B00103246F1
:101EE00000E033410090353C001037370070383245
:101EF00000A0392D00B03A2800A03B2300603C1E12
:101F000000103D1900903D1400103E0F00703E0A75
:101F100000C03E0500003F0000403FFBFF803FF651
:101F2000FFC03FF1FF46696C2E204469612E0046D8
:101F3000696C2E204469612E004520696E206D6D0C
:101F400033004F6666004F6E2000416476616E6319
:101F500065204B00416476616E6365204B00436FE2
:101F60006E74726F6C0050726F6265205A204F66FB
:101F70006673657400436F6E74726F6C00504944F1
:101F80002D44005049442D44005049442D490050EF
:101F900049442D49005049442D50005049442D508A
:101FA00000200220466163740020022046616374B1
:101FB000002002204D6178002002204D6178002031
:101FC00002204D696E002002204D696E004175743B
:101FD0006F74656D70004F6666004F6E200046613D
:101FE0006E2073706565640046616E207370656570
:101FF000640042656400426564004E6F7A7A6C65E5
:10200000004E6F7A7A6C6500436F6E74726F6C006D
:10201000526573746F7265206661696C7361666581
:10202000004C6F61642073657474696E677300534C
:10203000746F72652073657474696E67730044729F
:1020400069766520537472656E6774680046696CC2
:10205000616D656E74004D6F74696F6E0054656DCF
:102060007065726174757265004D61696E004578C6
:10207000747275646572004D6F7665205A004D6FFD
:1020800076652059004D6F76652058005072657056
:10209000617265004D6F766520302E316D6D004D9B
:1020A0006F766520316D6D004D6F76652031306D36
:1020B0006D004D6F766520617869730045787472A4
:1020C00075646572004D6F7665205A004D6F7665B8
:1020D0002059004D6F7665205800457874727564FC
:1020E0006572004D6F7665205A004D6F76652059F8
:1020F000004D6F76652058005072656865617420E8
:10210000414253005072656865617420504C410033
:10211000436F6F6C646F776E0044697361626C65C6
:10212000207374657070657273004D3834004265B9
:1021300064204C6576656C696E67004175746F202C
:10214000686F6D6500473238004D6F7665206178A5
:102150006973004D61696E0053746F726520736519
:102160007474696E6773004C6F6164207365747476
:10217000696E67730050726F6265205A204F666601
:1021800073657400426564204C6576656C696E67A2
:10219000004F6666004F6E20004C6576656C2062CD
:1021A0006564004732380A47323900473239004106
:1021B00075746F20686F6D65004732380050726526
:1021C00070617265005072656865617420414253A8
:1021D0002042656400507265686561742041425315
:1021E00020456E64005072656865617420414253F9
:1021F0000050726570617265005072656865617447
:1022000020504C41204265640050726568656174DD
:1022100020504C4120456E640050726568656174C1
:1022200020504C410050726570617265004441431A
:1022300020454550524F4D20577269746500452026
:10224000447269766572202500452044726976657E
:10225000722025005A204472697665722025005A42
:10226000204472697665722025005920447269768F
:102270006572202500592044726976657220250018
:10228000582044726976657220250058204472698E
:10229000766572202500436F6E74726F6C00507209
:1022A0006F6265205A204F666673657400466C6FD6
:1022B0007700466C6F770046616E207370656564C9
:1022C0000046616E2073706565640042656400427B
:1022D0006564004E6F7A7A6C65004E6F7A7A6C6531
:1022E000005370656564005370656564004D6169F5
:1022F0006E00436F6E74726F6C0050726570617225
:10230000650054756E6500437573746F6D20436F7F
:102310006D6D616E647300496E666F2073637265E4
:10232000656E00486F6D65202620496E666F004817
:10233000656174204265642F486F6D652F4C65762A
:10234000656C005072656865617420666F7220412B
:102350004253005072656865617420666F72205048
:102360004C4100486F6D6520262055424C20496E37
:10237000666F004D61696E004732380A4D35303363
:102380000A4D31313720557365722053637269707D
:102390007420446F6E65004D31343020533131303C
:1023A0000A4732380A4732390A4D313137205573DE
:1023B00065722053637269707420446F6E65004DBE
:1023C00031343020533131300A4D313034205332E2
:1023D00034300A4D313137205573657220536372A2
:1023E00069707420446F6E65004D3134302053376E
:1023F000300A4D31303420533138300A4D313137C5
:1024000020557365722053637269707420446F6E37
:1024100065004732380A47323920570A4D31313783
:1024200020557365722053637269707420446F6E17
:1024300065003344205072696E7465722052656184
:1024400064792E005072696E74696E672E2E2E00AC
:102450005072696E74207061757365640025753AF9
:102460002530327500253032753A2530327500201E
:102470002020200020202020202000040E1F041CEB
:10248000000000000E1315110E00001C1018170597
:10249000060500040A0A0A0A11110E0C12120C0099
:1024A000000000001F1511151F000050726F6265BB
:1024B000205A204F666673657400506C65617365C1
:1024C000207265736574005052494E54455220483D
:1024D000414C5445440001290229042908291029A6
:1024E000202940298029012C022C012602260426BD
:1024F00008261026202640268026402C802C0123EA
:1025000002230423082310232023402380230120B7
:102510000220042008201020202040208020102CA1
:10252000202C012F022F042F082F102F202F402F97
:10253000802F7EFE7EFD7EFB7EF77EEF7EDF7EBF00
:102540007E7F00010000F3251200020000B0254349
:1025500000030000AC2504010309049225180203BE
:1025600009047A2516030309046C250C0C033100B9
:1025700032003300340035000000160355005300CC
:1025800042002000530065007200690061006C0089
:10259000000018035400650065006E0073007900A8
:1025A0006400750069006E006F00000004030904F8
:1025B00009024300020100C03209040000010202C6
:1025C0000100052400100105240100010424020675
:1025D00005240600010705820308004009040100E4
:1025E000020A0000000705030240000007058402FC
:1025F0004000001201000202000020C01683047295
:1026000002010203010001C102018036018136008E
:10261000BE5DF478C2A25DC959DAC75D11241FBE40
:10262000CFEFD0E2DEBFCDBF12E0A0E0B1E0E4E149
:10263000FDEC01E00BBF02C007900D92AA36B10776
:10264000D9F72FE0AAE6B2E001C01D92A634B20786
:10265000E1F713E1CDE0D3E104C02197FE010E9430
:10266000EDDAC830D107C9F70E94E8D10C947DE6B5
:102670000C9400004F925F926F927F928F929F9284
:10268000AF92BF92CF92DF92EF92FF92CF934B0126
:102690005C0169017A0120E030E040EA51E40E94E7
:1026A00015DB2B013C012FE632E143E85AEB0E9497
:1026B000F2DD87FD48C023E830E048EC52E4C30176
:1026C000B2010E94EFDB18160CF43DC02FE632E198
:1026D00043E85AEBC701B6010E94F2DD87FD33C023
:1026E00023E830E048EC52E4C701B6010E94EFDB7A
:1026F00018164CF124EF3DEF4FE951E4C501B40148
:102700000E94F2DD87FD1FC023E830E044EB52E475
:10271000C501B4010E94EFDB1816ACF027EE3BEFC9
:102720004FE151E4C701B6010E94F2DD87FD0BC005
:10273000C1E023E830E044EB52E4C701B6010E9457
:10274000EFDB18160CF4C0E08C2FCF91FF90EF90C8
:10275000DF90CF90BF90AF909F908F907F906F90C1
:102760005F904F900895FB0101900020E9F73197A9
:10277000AF01461B570BDC01ED91FC910280F38108
:10278000E02D0994CF93DF931F92CDB7DEB7698315
:10279000DC01ED91FC910280F381E02D41E050E0FD
:1027A000BE016F5F7F4F09950F90DF91CF91089524
:1027B000FF920F931F93CF93DF93F82E092F162FBD
:1027C000E0EAF4E06491EF012196662329F088E3C2
:1027D0009FE0D8DFFE01F6CFEF2DF02F6491EF01DF
:1027E0002196662329F088E39FE0CCDFFE01F6CF37
:1027F000EEE9F4E06491EF012196662329F088E385
:102800009FE0C0DFFE01F6CF412F50E060E070E0B6
:1028100088E39FE00E94EED06AE088E39FE0DF91CA
:10282000CF911F910F91FF90ADCF0FB6F89480918B
:102830002D0F90912E0FA0912F0FB091300F0FBE42
:102840008093E9029093EA02A093EB02B093EC022A
:1028500008954F925F926F927F92AF92BF92CF9204
:10286000DF92EF92FF92CF93DF93EB01FC01608147
:102870007181828193812CE3C22ED12CE12CF12C29
:10288000A70196010E94AFDAB62EA72ECA01B901A0
:10289000A70196010E94AFDA6B017C01CA01B90160
:1028A00028E130E040E050E00E94AFDA2B013C012B
:1028B000C9016DE671E00E9488DA61157105D9F0F1
:1028C000AF92BF92DF92CF925F924F929F938F937E
:1028D0007F936F938CE497E09F938F93DF93CF93D5
:1028E0000E9463E38DB79EB70E960FB6F8949EBF15
:1028F0000FBE8DBF61C00097C9F0AF92BF92DF924B
:10290000CF925F924F929F938F938CE397E09F9328
:102910008F93DF93CF930E9463E3EDB7FEB73C96AE
:102920000FB6F894FEBF0FBEEDBF46C04114510470
:1029300061047104B9F0AF92BF92DF92CF925F92BF
:102940004F9280E397E09F938F93DF93CF930E9402
:1029500063E38DB79EB70A960FB6F8949EBF0FBE7D
:102960008DBF2AC0C114D104E104F104A9F0AF92D3
:10297000BF92DF92CF9288E297E09F938F93DF938D
:10298000CF930E9463E3EDB7FEB738960FB6F89485
:10299000FEBF0FBEEDBF10C0AF92BF9284E297E0C2
:1029A0009F938F93DF93CF930E9463E30F900F90D9
:1029B0000F900F900F900F90DF91CF91FF90EF90BD
:1029C000DF90CF90BF90AF907F906F905F904F90CF
:1029D000089581548A3108F040C0A82FB0E040919A
:1029E000210550912205609123057091240504C0B2
:1029F00076956795579547958A95D2F740FF2DC0F4
:102A0000E0912C05F0912D05A95FBA4F8C91882398
:102A1000E1F0E80FF11D808190ED980F9A3080F081
:102A20008E3229F4818180538A3078F409C08D3246
:102A300011F08B3251F4818190ED980F9A3018F497
:102A40009E2F8F2F04C08E3251F090E080E0909343
:102A500028058093290581E0089580E0089582810A
:102A600080538A3090F7ECCFB4DF882341F081E0C7
:102A70002091280530912905232B09F480E0089541
:102A80000F931F93CF93809128059091290500976C
:102A900011F1FC018F01C1912C2F2F7DA9F0C534BC
:102AA00011F0C536B9F7F801108260E070E080914E
:102AB0002805909129050E94F7DEF801C083562F62
:102AC000472F382F292F0BC060E070E0CF911F9166
:102AD0000F910C94F7DE50E040E030E020E0652FED
:102AE000742F832F922FCF911F910F910895809172
:102AF000280590912905009731F04AE050E060E008
:102B000070E00C945DE060E070E0CB01089580918E
:102B1000280590912905009731F04AE050E060E0E7
:102B200070E00C9485E160E070E0CB010895DFDF98
:102B300097FD0AC0DCDF6F3F71058105910509F043
:102B40002CF4D5DF862F089580E008958FEF089547
:102B50008091280590912905892B31F0E8DF91E0DB
:102B6000811103C090E001C091E0892F08950F9377
:102B70001F93CF93DF93CDB7DEB72C970FB6F894A2
:102B8000DEBF0FBECDBFEEECF4E080859185A2855F
:102B9000B3854481558166817781008111812281CD
:102BA000338109871A872B873C874D835E836F8328
:102BB000788789839A83AB83BC83AE014F5F5F4F75
:102BC000BE016B5F7F4FCE0109960E9403682AED1C
:102BD00034E0AE014F5F5F4FBE016B5F7F4FCE01B0
:102BE00009960E94A4762C960FB6F894DEBF0FBE0D
:102BF000CDBFDF91CF911F910F9108952F923F92FA
:102C00004F925F926F927F929F92AF92BF92CF92BC
:102C1000DF92EF92FF920F931F93CF93DF93CDB785
:102C2000DEB764970FB6F894DEBF0FBECDBF2A01A2
:102C30003B01902EA12E6901082F10E0F801E55804
:102C4000F54FE491BB24B3941E160CF4B12CFF2471
:102C5000F39420E030E0A901C301B2010E94F2DD4B
:102C600018160CF0F12C000F111F000F111FC801D6
:102C700082539B4F1C01FC0110821182128213822D
:102C800076DFF1014082518262827382E090F2022B
:102C900020E030E0A901692D7A2DC6010E94EFDB0A
:102CA000811108C0F801E654F54F85919591A591E1
:102CB000B49103C0892D9A2DD601898B9A8BAB8B49
:102CC000BC8B8091D6049091D704A091D804B09188
:102CD000D9044091D2045091D3046091D4047091EE
:102CE000D5040091CE041091CF042091D0043091EE
:102CF000D1040D871E872F87388B49875A876B87AA
:102D00007C878D839E83AF83B88719821A821B824A
:102D10001C82AE014B5F5F4FBE01675F7F4FCE01EC
:102D20000D960E940368CE0101966C018E010F5E24
:102D30001F4F2AED34E0AE014B5F5F4FBE01675F6E
:102D40007F4F0C960E94C2750E949F69BF100E941F
:102D5000C55B64960FB6F894DEBF0FBECDBFDF91A2
:102D6000CF911F910F91FF90EF90DF90CF90BF9088
:102D7000AF909F907F906F905F904F903F902F907B
:102D800008956AED74E083E00C94CA77CF93DF93E3
:102D900000D0CDB7DEB720912A0F30912B0FCE0196
:102DA00001962115310529F486549F409A83898321
:102DB00004C0821B930B9A83898389819A810F9027
:102DC0000F90DF91CF910895FF920F931F93CF93B0
:102DD000DF93FC0120812B3319F1D091B304D4305F
:102DE000F8F4F62EBC01C091B1040C2F10E0F0E60F
:102DF000CF9FC00111248F5C9C4F0E9434E3F801E7
:102E0000E053FD4FF082CF5FC43018F4C093B1049B
:102E100002C01092B104DF5FD093B30481E001C01F
:102E200080E0DF91CF911F910F91FF900895EF9275
:102E3000FF921F93CF93DF937C0160E0C5DF182FD3
:102E40008823C9F0E0E3F2E16491EF012196662363
:102E500029F088E39FE096DCFE01F6CFB7018EE60D
:102E60009AE00E94F87862E288E39FE08BDC6AE0F7
:102E700088E39FE087DC812FDF91CF911F91FF9046
:102E8000EF900895DF92EF92FF920F931F93CF93ED
:102E9000DF93CDB7DEB76E970FB6F894DEBF0FBEE7
:102EA000CDBF60912F03709130036115710541F121
:102EB0004DE150E0CE0101967C010E94E3E21E8EBE
:102EC000F7018F010E191F09D190DD2019F09AE04A
:102ED000D912F7CFF701E00FF11F1082C701A7DF6A
:102EE000882371F0DD20A9F00F5F1F4F80912F0321
:102EF00090913003080F191F1093300300932F0394
:102F000081E020912F0330913003232B29F480E0BE
:102F100003C000E010E0F0CF6E960FB6F894DEBF6D
:102F20000FBECDBFDF91CF911F910F91FF90EF901A
:102F3000DF9008959093300380932F03A3CFEF92F7
:102F4000FF920F931F93CF93DF937C0184E58CDD79
:102F5000D82F882369F1EBDDC82F18162CF5E0E394
:102F6000F2E164918F010F5F1F4F662329F088E320
:102F70009FE008DCF801F5CF6DE488E39FE002DC18
:102F8000A70160E070E020E088E39FE00E9492D01B
:102F90006C2FCC0F770B80E599E00E9420796AE0D6
:102FA00088E39FE0EFDB08C08093E402D0E004C038
:102FB0008091F2028093E4028D2FDF91CF911F91D7
:102FC0000F91FF90EF9008950F931F93CF93DF938E
:102FD00094E0899FE00111248E010F5F1C4FFE01D8
:102FE000E35FFC4FDE01A75EBC4F2D913D914D91FB
:102FF0005C9160817181828193810E9416DBF8016E
:103000006083718382839383FE01E255F54F85913E
:103010009591A591B491FE01EB50FD4F8083918372
:10302000A283B383FE01EE55F54F85919591A5914D
:10303000B491C55FDE4F88839983AA83BB83DF91F8
:10304000CF911F910F910895CF92DF92EF920F933E
:103050001F93CF93DF93CDB7DEB760970FB6F89489
:10306000DEBF0FBECDBFE090F202EEECF4E0808553
:103070009185A285B38544815581668177810081E0
:103080001181228133810D871E872F87388B4987D5
:103090005A876B877C878D839E83AF83B88719821D
:1030A0001A821B821C82AE014B5F5F4FBE01675FBD
:1030B0007F4FCE010D960E940368CE0101966C01F0
:1030C00009E111E02AED34E0AE014B5F5F4FBE0134
:1030D000675F7F4F0C960E94C27560960FB6F8949A
:1030E000DEBF0FBECDBFDF91CF911F910F91EF904B
:1030F000DF90CF9008954F925F926F927F928F9260
:103100009F92AF92BF92CF92DF92EF92FF920F9376
:103110001F93CF93DF93CDB7DEB72C970FB6F894FC
:10312000DEBF0FBECDBF6D837E838F8398872987D7
:103130003A874B875C874701580136018091190116
:1031400090911A01A0911B01B0911C0189839A836F
:10315000AB83BC83D601CD90DD90ED90FC9020E058
:1031600030E0A901C701B6010E94EFDB811106C062
:10317000E2ECFAE0C590D590E590F490A5019401B9
:103180006091D6047091D7048091D8049091D904AD
:103190000E94EFDB87FF11C0C0921901D0921A0183
:1031A000E0921B01F0921C018092D6049092D70409
:1031B000A092D804B092D90447DFF3014080518037
:1031C0006280738020E030E0A901C301B2010E9457
:1031D000EFDB811108C04090010150900201609026
:1031E0000301709004014092190150921A016092FB
:1031F0001B0170921C018D819E81AF81B8858093E7
:10320000CE049093CF04A093D004B093D1048985C9
:103210009A85AB85BC858093D2049093D304A09308
:10322000D404B093D50410DFA50194016091D604B5
:103230007091D7048091D8049091D9040E94F2DD56
:1032400018168CF4C0921901D0921A01E0921B0159
:10325000F0921C018092D6049092D704A092D804D8
:10326000B092D904F1DE0E949F6989819A81AB8175
:10327000BC818093190190931A01A0931B01B09314
:103280001C012C960FB6F894DEBF0FBECDBFDF91A8
:10329000CF911F910F91FF90EF90DF90CF90BF9053
:1032A000AF909F908F907F906F905F904F90089518
:1032B000CF92DF92EF92FF920F931F936B01FC016D
:1032C000E080F18002811381EEECF4E0248135810D
:1032D0004681578160817181828193810CDF1F91CA
:1032E0000F91FF90EF90DF90CF900895CF92DF92F3
:1032F000EF92FF920F931F936A01E090D604F09033
:10330000D7040091D8041091D904FB0120813181A8
:1033100042815381FC016081718182819381EBDE66
:103320001F910F91FF90EF90DF90CF9008958091C3
:10333000190190911A01A0911B01B0911C01809379
:103340002B0390932C03A0932D03B0932E03809115
:1033500017019091180190932A038093290384E622
:1033600090E09093180180931701089580912B03AA
:1033700090912C03A0912D03B0912E0380931901FD
:1033800090931A01A0931B01B0931C018091290313
:1033900090912A0390931801809317010895EF925A
:1033A000FF921F93CF93DF93882329F0D091BD0420
:1033B000D095D17001C0D0E0662341F01091BD04DA
:1033C00011FB882780F911E0182701C010E0442381
:1033D00041F0C091BD04C2FB882780F9C1E0C82735
:1033E00001C0C0E0D11105C0111103C0CC2309F404
:1033F00086C0E0E3F2E164917F018FEFE81AF80AFA
:10340000662329F088E39FE0BDD9F701F4CFEAE411
:10341000F9E064917F019FEFE91AF90A662329F028
:1034200088E39FE0AFD9F701F4CFDD2371F0E8E442
:10343000F9E064917F018FEFE81AF80A662329F01A
:1034400088E39FE09FD9F701F4CF112371F0E6E400
:10345000F9E064917F019FEFE91AF90A662329F0E8
:1034600088E39FE08FD9F701F4CFC11103C0ECE3EB
:10347000F9E00EC0E4E4F9E064917F018FEFE81A0F
:10348000F80A6623A1F388E39FE07CD9F701F4CF23
:1034900064917F019FEFE91AF90A662329F088E316
:1034A0009FE070D9F701F4CFC11103C04EEE51E097
:1034B00002C04EED51E0111103C02EEE31E002C00A
:1034C00020EE31E0D11103C08EEE91E002C082EE19
:1034D00091E05F934F933F932F939F938F938AE253
:1034E00099E09F938F931F920E945DA08DB79EB726
:1034F00009960FB6F8949EBF0FBE8DBFC1E08C2F0A
:10350000DF91CF911F91FF90EF900895BF92CF92DE
:10351000DF92EF92FF920F931F93CF93DF93CDB77C
:10352000DEB728970FB6F894DEBF0FBECDBF9091DF
:10353000EA04981709F47AC0B82E882309F453C016
:1035400080E090E0A0EAB0E48D839E83AF83B887EB
:10355000C090E002D090E102E090E202F090E3023D
:1035600020E030E0A901C701B6010E94EFDB87FF30
:103570000CC0A701960160E070E080EA90E40E9430
:1035800015DB6D837E838F83988720E030E043E0F6
:1035900053E46D817E818F8198850E94F2DD18163B
:1035A00044F480E090E0A3E0B3E48D839E83AF8396
:1035B000B8872091D6043091D7044091D804509117
:1035C000D9046D817E818F8198850E94F2DD181665
:1035D00054F419821A821B821C82BE016F5F7F4FD6
:1035E000CE01059665DE6091CE047091CF04809186
:1035F000D0049091D1042091D2043091D304409111
:10360000D4045091D50419821A821B821C82E09046
:10361000D604F090D7040091D8041091D904FE018B
:1036200031966F0168DD8B2D0E94D05B80E028967B
:103630000FB6F894DEBF0FBECDBFDF91CF911F91C3
:103640000F91FF90EF90DF90CF90BF9008954F9231
:103650005F926F927F928F929F92AF92BF92CF9222
:10366000DF92EF92FF920F931F93CF93C82FE82E14
:10367000F12CF701E558F54FB490823021F481E048
:1036800045DF811107C16701CC0CDD1CCC0CDD1CB2
:10369000F601E657F54F45905590659074906B2D67
:1036A000BB0C770B880B990B0E9491DC4B015C01E2
:1036B00020E030E040EC5FE3C301B2010E942DDE68
:1036C000A50194010E942DDEAB01BC0100E010E0D9
:1036D00098018C2F93DAC23041F0F601E258F54F91
:1036E000259135914591549104C020E030E040E4AB
:1036F00050E4C501B4010E942DDE4B015C0120E0C5
:1037000030E0A9010E94EFDB882309F45CC0C230DD
:1037100021F000E010E0980104C000E010E020E893
:1037200030E4B501A40170588C2F68DAC23009F476
:1037300039C0F701EB54F74F849181111DC0E0E3CC
:10374000F2E164917F018FEFE81AF80A662329F00D
:1037500088E39FE017D8F701F4CFE3E9F8E064913C
:103760007F018FEFE81AF80A662329F088E39FE0CB
:1037700009D8F701F4CF8AE0F601E654F54F4590F9
:10378000559065907490682F70E080E090E00E9402
:1037900091DC9B01AC01C301B2010E94F6DB2B015D
:1037A0003C0105C0412C512C612C90E4792EA501DF
:1037B0009401C501B4010E9416DBAB01BC01930169
:1037C00082018C2F1BDA81E090E00C2E01C0880F63
:1037D0000A94EAF79091BC04982B9093BC049091C2
:1037E000BD04892B8093BD04F601E75EFC4F108277
:1037F0001182128213828C2FE7DBF601EA56F54F15
:1038000085919591A591B491F601E253FB4F808388
:103810009183A283B383C230D1F42091E00230912E
:10382000E1024091E2025091E3026091D60470916E
:10383000D7048091D8049091D9040E9415DB60933D
:10384000D6047093D7048093D8049093D9048FD969
:10385000F601E254FB4FD601A253BB4F8D919D91CF
:103860000D90BC91A02D80839183A283B383C2303D
:1038700089F480E0CF911F910F91FF90EF90DF903E
:10388000CF90BF90AF909F908F907F906F905F9000
:103890004F903CCECF911F910F91FF90EF90DF9012
:1038A000CF90BF90AF909F908F907F906F905F90E0
:1038B0004F90089581E00895AF92BF92CF92DF922A
:1038C000EF92FF920F931F93CF93DF9382E0A82E86
:1038D00082E0B82E9EEBE92E94E0F92E0EEC14E077
:1038E00021E0C22E23E0D22EC0E0D0E0F50181918C
:1038F0005F016FD8882319F1C3D8FE01EB5DFC4F3F
:103900002081211104C02091F102222341F0F8010D
:1039100020813181428153810E9416DB0AC0C3306D
:10392000D10539F0F60120813181428153810E9415
:1039300015DBF70160837183828393830AC0F801EA
:1039400080819181A281B381F70180839183A283D9
:10395000B3832196F4E0EF0EF11C0C5F1F4F84E05F
:10396000C80ED11CC430D10509F0C0CF86E47CD884
:103970008823B9F085D820E030E0A9010E94F2DD6B
:1039800018167CF47DD820E030E040E752E40E9435
:10399000F6DB6093190170931A0180931B019093D9
:1039A0001C01DF91CF911F910F91FF90EF90DF905D
:1039B000CF90BF90AF900895CF92DF92EF92FF9299
:1039C0000F931F93CF93DF930FB6F894C0902D0FF2
:1039D000D0902E0FE0902F0FF090300F0FBE8091FF
:1039E000EF02811174C080910001882309F46FC037
:1039F0008091CF02882309F46AC04091CB02509194
:103A0000CC026091CD027091CE0297018601041B19
:103A1000150B260B370B37FD6DC0833031F134F4B5
:103A200081300CF454C0E0E3F2E106C0843009F0C8
:103A30004EC0E0E3F2E133C06491EF0121966623CA
:103A400031F088E39FE00E94C213FE01F5CFE7EE5C
:103A5000F8E06491EF012196662309F438C088E309
:103A60009FE00E94C213FE01F4CFE0E3F2E1649113
:103A7000EF012196662331F088E39FE00E94C21394
:103A8000FE01F5CFE0EDF8E06491EF0121966623A9
:103A9000F1F088E39FE00E94C213FE01F5CF64912C
:103AA000EF012196662331F088E39FE00E94C21364
:103AB000FE01F5CFE8EBF8E06491EF012196662373
:103AC00031F088E39FE00E94C213FE01F5CF209100
:103AD000000130E0A8EEB3E00E94F6DAC60ED71E71
:103AE000E81EF91EC092CB02D092CC02E092CD0229
:103AF000F092CE02DF91CF911F910F91FF90EF9046
:103B0000DF90CF9008950F931F93CF93DF9300D052
:103B100000D0CDB7DEB78091BC048370833011F143
:103B200060E085E898E00E9413A0E0E3F2E1649190
:103B30008F010F5F1F4F662331F088E39FE00E94E3
:103B4000C213F801F4CFE6E7F8E064918F010F5F4C
:103B50001F4F662309F43DC088E39FE00E94C21313
:103B6000F801F3CF04D880E090E0A8E4B2E48093B9
:103B7000C2049093C304A093C404B093C50480917D
:103B8000D6049091D704A091D804B091D904809321
:103B9000C6049093C704A093C804B093C90480E0FE
:103BA00090E0A0EFB1E48093BE049093BF04A09393
:103BB000C004B093C10419821A821B821C82AE0118
:103BC0004F5F5F4F62EC74E08EEB94E08FDB82E03E
:103BD0003EDD0F900F900F900F90DF91CF911F91CE
:103BE0000F9108950F931F93CF93DF93CDB7DEB757
:103BF00069970FB6F894DEBF0FBECDBF0E94138940
:103C00006E8B7F8B888F998FBE016F5F7F4FCE0148
:103C100046960E94291460E0CE0101960E94EC9F16
:103C2000E0E3F2E164918F010F5F1F4F662331F0F3
:103C300088E39FE00E94C213F801F4CFBE016F5FDA
:103C40007F4F80E697E00E94F8786AE088E39FE083
:103C50000E94C21369960FB6F894DEBF0FBECDBFA7
:103C6000DF91CF911F910F910895CF93DF93E6E3FA
:103C7000F2E16491EF012196662331F088E39FE041
:103C80000E94C213FE01F5CFE8EEF6E06491EF0169
:103C90002196662331F088E39FE00E94C213FE0163
:103CA000F5CFDF91CF91089588E690E048D9811152
:103CB00024C08091DE0483FD20C083E50E9434157A
:103CC0008823C9F00E9440150E945EDC7093B10DFC
:103CD0006093B00D80E00E94718D0E94401520E03D
:103CE00030E04AEA52E40E94EFDB181624F00E940A
:103CF000BC880E944DA00C94C4780895CF93DF93A4
:103D000089E690E01CD9811116C0EAE9F6E06491D9
:103D1000EF012196662331F088E39FE00E94C213F1
:103D2000FE01F5CF0E9427936AE088E39FE0DF91D0
:103D3000CF910C94C213DF91CF910895CF92DF926F
:103D4000EF92FF9283E50E943415882321F10E94AF
:103D500097158D3308F08CE38093460D0FB6F894D9
:103D6000C0902D0FD0902E0FE0902F0FF090300FBD
:103D70000FBE282F30E0A8EEB3E00E94F6DAC60EA0
:103D8000D71EE81EF91EC092420DD092430DE0925C
:103D9000440DF092450DFF90EF90DF90CF90089585
:103DA00080E50E943415811106C083E50E94341518
:103DB000882359F005C00E94971581110CC0F5CFDA
:103DC0000E9477156F3F710510F06FEF70E07093F0
:103DD000F4026093F30208958091DE0483FD14C021
:103DE00083E50E943415882379F00E9440150E94D3
:103DF0005EDC6639710514F066E970E07093A90D18
:103E00006093A80D0C94C38D0895DF92EF92FF92FA
:103E10000F931F93CF93DF9383E50E94E9148823C8
:103E200059F083E50E943415882319F00E949715F4
:103E300001C080E08093DE04E0E3F2E16491EF01F1
:103E40002196662331F088E39FE00E94C213FE01B1
:103E5000F5CFE1EEF6E06491EF012196662331F0B3
:103E600088E39FE00E94C213FE01F5CF8091DE043B
:103E70008823A9F187EDE82E86E0F82E00E010E017
